:100000000C9462000C948A000C948A000C948A0070
:100010000C948A000C948A000C948A000C948A0038
:100020000C948A000C948A000C948A000C948A0028
:100030000C948A000C948A000C948A000C948A0018
:100040000C941F020C948A000C948A000C948A0071
:100050000C948A000C948A000C948A000C948A00F8
:100060000C948A000C948A000000000024002700F1
:100070002A0000000000250028002B0000000000DE
:1000800023002600290004040404040404040202DA
:100090000202020203030303030301020408102007
:1000A0004080010204081020010204081020000012
:1000B0000008000201000003040700000000000027
:1000C00000004C0511241FBECFEFD8E0DEBFCDBF2E
:1000D00011E0A0E0B1E0E2E1FFE002C005900D9286
:1000E000AA30B107D9F721E0AAE0B1E001C01D9222
:1000F000A637B207E1F710E0C2E6D0E004C02197CE
:10010000FE010E948107C136D107C9F70E9469022A
:100110000C9487070C94000080916D0190916E0102
:10012000A0916F01B0917001EBE2F1E02BE431E0BE
:10013000AC01BD01032E3DE0440F551F661F771F24
:100140003A95D1F7302D84279527A627B727AC01FC
:10015000BD01032E31E176956795579547953A9500
:10016000D1F7302D84279527A627B727AC01BD01ED
:10017000689414F8440F551F661F771F1694D1F723
:1001800084279527A627B7278193AC01BD01032EAD
:100190003DE0440F551F661F771F3A95D1F7302D6C
:1001A00084279527A627B727AC01BD01032E31E18F
:1001B00076956795579547953A95D1F7302D8427D1
:1001C0009527A627B727AC01BD01689414F8440F02
:1001D000551F661F771F1694D1F784279527A627EA
:1001E000B727878F2E173F0709F0A2CF80936D01A5
:1001F00090936E01A0936F01B093700108958330C6
:1002000081F028F4813099F08230A9F00895873088
:10021000A9F08830C9F08430B1F4809180008F7DDE
:1002200003C0809180008F7780938000089584B50B
:100230008F7784BD089584B58F7DFBCF8091B0000A
:100240008F778093B00008958091B0008F7DF9CFB3
:10025000CF93DF93282F30E0F901E255FF4F8491CF
:10026000F901E656FF4FD491F901EA57FF4FC491C7
:10027000CC23A1F081110E94FF00EC2FF0E0EE0FE3
:10028000FF1FE458FF4FA591B491EC91ED2381E05D
:1002900090E009F480E0DF91CF91089580E090E054
:1002A000FACF1F93CF93DF93282F30E0F901E25567
:1002B000FF4F8491F901E656FF4FD491F901EA57B7
:1002C000FF4FC491CC23A9F0162F81110E94FF008B
:1002D000EC2FF0E0EE0FFF1FEE58FF4FA591B49109
:1002E0008FB7F894EC91111108C0D095DE23DC9300
:1002F0008FBFDF91CF911F910895DE2BF8CFCF9361
:10030000DF9390E0FC01E656FF4F24918A579F4F00
:10031000FC0184918823D1F090E0880F991FFC01A3
:10032000E859FF4FA591B491FC01EE58FF4FC591DC
:10033000D491623071F49FB7F8943C91822F8095EC
:1003400083238C93E8812E2B28839FBFDF91CF914D
:1003500008958FB7F894EC912E2B2C938FBFF6CF86
:100360001F93CF93DF93182FEB0161E00E947F0171
:10037000209739F460E0812FDF91CF911F910C9489
:100380005101CF3FD10511F461E0F5CFE12FF0E04D
:10039000E255FF4FE491E33031F140F4E130B1F048
:1003A000E230E1F0C038D1057CF7E4CFE73029F145
:1003B000E83059F1E430B1F7809180008062809399
:1003C0008000D0938B00C0938A0004C084B58068FD
:1003D00084BDC7BDDF91CF911F91089584B5806220
:1003E00084BDC8BDF7CF8091800080688093800075
:1003F000D0938900C0938800EDCF8091B0008068D1
:100400008093B000C093B300E5CF8091B0008062CC
:100410008093B000C093B400DDCF8E508064809391
:100420007C0080917A00806480937A0080917A00C9
:1004300086FDFCCF809178009091790008951F92FD
:100440000F920FB60F9211242F933F938F939F9388
:10045000AF93BF938091270190912801A09129012A
:10046000B0912A013091260123E0230F2D3758F552
:100470000196A11DB11D2093260180932701909321
:100480002801A0932901B0932A0180912201909123
:100490002301A0912401B09125010196A11DB11D58
:1004A0008093220190932301A0932401B09325010E
:1004B000BF91AF919F918F913F912F910F900FBE60
:1004C0000F901F90189526E8230F0296A11DB11DCD
:1004D000D2CFCF93DF93CDB7DEB72A970FB6F8947C
:1004E000DEBF0FBECDBF789484B5826084BD84B575
:1004F000816084BD85B5826085BD85B5816085BD1F
:1005000080916E00816080936E00109281008091D6
:10051000810082608093810080918100816080935E
:100520008100809180008160809380008091B10083
:1005300084608093B1008091B00081608093B000AE
:1005400080917A00846080937A0080917A00826042
:1005500080937A0080917A00816080937A00809104
:100560007A00806880937A001092C10062E084E093
:100570000E947F0161E083E00E947F0161E08BE0E7
:100580000E947F0162E081E10E947F0161E08AE0D8
:100590000E947F0162E089E00E947F0183E28093F4
:1005A000B00081E08093B10082E88093800089E10F
:1005B000809381008FEF90E0909387008093860076
:1005C00060E08BE00E9451018EE00E940D02092E36
:1005D000000CAA0BBB0B0097A105B10521F481E02B
:1005E00090E0A0E0B0E080936D0190936E01A09345
:1005F0006F01B09370010E948C0010926B011092F9
:100600007101109272011092730110927401109294
:1006100075018EE00E940D02E0E087369105A4F09E
:10062000E1E0853321E092077CF0E2E0833032E0C4
:10063000930754F0E3E0813D42E094072CF0E4E0BE
:100640008F3993400CF0E5E0F0E0ED5FFE4F8081E4
:1006500080936C0101E012E08FB7F894209127019C
:10066000309128014091290150912A0129833A8330
:100670004B835C838FBF20931E0130931F014093F7
:1006800020015093210181E10E9428011C01019762
:1006900009F027C180910201811123C180E10E94EC
:1006A0000D02BC01990F880B990B0E942B0620E0CC
:1006B00030EC4FE754E40E9481056B017C018FE030
:1006C0000E940D02BC01990F880B990B0E942B060A
:1006D00020E030EC4FE754E40E9481054B015C01BF
:1006E0008EE00E940D02BC01990F880B990B0E94AD
:1006F0002B0620E030EC4FE754E40E9481052B01EB
:100700003C012DE033E34CEC5DE30E947C05E0E02E
:1007100018166CF52AE836E24AE95EE3C301B20135
:100720000E947C05E1E0181614F528E230EA40E06A
:100730005FE3C301B2010E947C05E2E01816BCF43D
:100740002BE03DE244E35FE3C301B2010E947C057C
:10075000E3E0181664F42EEE39EB47E65FE3C301DD
:10076000B2010E947C05E4E018160CF4E5E0F0E02C
:10077000ED5FFE4F40814D8320E030E0A901C501CF
:10078000B4010E947C0587FD5DC120E030E040E8B7
:100790005FE3C501B4010E94DB06181634F4812C16
:1007A000912C90E8A92E9FE3B92E20E030E0A9011A
:1007B000C701B6010E947C0587FD48C120E030E0FA
:1007C00040E85FE3C701B6010E94DB06181634F467
:1007D000C12CD12C80E8E82E8FE3F82E80916C019B
:1007E0005D81851761F080916B01851728F0652F79
:1007F0000E944D0790936B018D8180936C018091D5
:100800006B0190E0019660916C0170E00E945907C5
:1008100080936B01DC01A55DBE4FBA87A9876C91FF
:1008200070E090E080E00E942B0620E030E04FE78F
:1008300053E40E9481056D837E838F839887609344
:100840007101709372018093730190937401E98533
:10085000FA8560A170E090E080E00E94290620E027
:1008600030E04FE753E40E9481052B013C01A701D2
:1008700096010E947C05881F8827881F8093750138
:10088000A50194016D817E818F8198850E94E0068B
:1008900020E030E04FE753E40E94E0060E94F305B9
:1008A0004B018AE00E94B001B40183E00E94B001D4
:1008B000A7019601C301B2010E947C0587FFCAC04F
:1008C00089819A81AB81BC810A96A11DB11D80935B
:1008D0001A0190931B01A0931C01B0931D0110926B
:1008E000010181E0232809F480E08093020189E07E
:1008F0000E9428019A838983019791F480910001D5
:1009000081110EC00E948C0010926B011092710137
:10091000109272011092730110927401109275017D
:1009200081E029813A81232B09F480E08093000142
:1009300080910101C0901E01D0901F01E090200124
:10094000F0902101811189C080911A0190911B01C1
:10095000A0911C01B0911D01A7019601281B390B24
:100960004A0B5B0BDA01C901B7FD0EC061E08BE0F9
:100970000E945101C0921601D0921701E092180115
:10098000F09219010093010184E00E942801109265
:1009900014011092150190911301891751F0809361
:1009A0001301C0920E01D0920F01E0921001F0925B
:1009B000110180910E0190910F01A0911001B09151
:1009C0001101C81AD90AEA0AFB0A80910A0190911A
:1009D0000B01A0910C01B0910D018C159D05AE0588
:1009E000BF05B0F49091120180911301981781F026
:1009F00080931201911103C021E0813009F020E0C1
:100A000020931401913009F4811190E09093150125
:100A100080911501882371F00E948C0010926B0167
:100A20001092710110927201109273011092740170
:100A30001092750140E050E0452B09F40DCE0E9464
:100A400000000ACE812C912C5401AFCEC12CD12CA8
:100A50007601C4CE1093010144CF813009F094CFC8
:100A60008091160190911701A0911801B091190180
:100A7000A7019601281B390B4A0B5B0BDA01C90150
:100A80000397A105B10508F47FCF60E08BE00E94D9
:100A900051011093010178CFEAE0F1E082E390E0A8
:100AA000A0E0B0E080839183A283B3831482158297
:100AB0001682178281E080878187128613861092C2
:100AC0006B0188E080936C018FEE9EEBADEABEED8A
:100AD00080936D0190936E01A0936F01B0937001AC
:100AE00010927101109272011092730110927401B0
:100AF000109275010C948C000E94660608F481E047
:100B000008950E9495050C94A1060E949A0658F03B
:100B10000E94930640F029F45F3F29F00C948A0666
:100B200051110C94D5060C9490060E94B20668F3FD
:100B30009923B1F3552391F3951B550BBB27AA2796
:100B400062177307840738F09F5F5F4F220F331FD0
:100B5000441FAA1FA9F335D00E2E3AF0E0E832D098
:100B600091505040E695001CCAF72BD0FE2F29D09B
:100B7000660F771F881FBB1F261737074807AB076D
:100B8000B0E809F0BB0B802DBF01FF2793585F4FE2
:100B90003AF09E3F510578F00C948A060C94D506E5
:100BA0005F3FE4F3983ED4F3869577956795B795C4
:100BB000F7959F5FC9F7880F911D9695879597F9CF
:100BC0000895E1E0660F771F881FBB1F6217730748
:100BD0008407BA0720F0621B730B840BBA0BEE1F5D
:100BE00088F7E09508950E94FA056894B1110C9475
:100BF000D50608950E94BA0688F09F5798F0B92F3D
:100C00009927B751B0F0E1F0660F771F881F991F41
:100C10001AF0BA95C9F714C0B13091F00E94D40609
:100C2000B1E008950C94D406672F782F8827B85F19
:100C300039F0B93FCCF3869577956795B395D9F799
:100C40003EF490958095709561957F4F8F4F9F4FA3
:100C50000895E89409C097FB3EF4909580957095AF
:100C600061957F4F8F4F9F4F9923A9F0F92F96E9F8
:100C7000BB279395F695879577956795B795F1116D
:100C8000F8CFFAF4BB0F11F460FF1BC06F5F7F4F0A
:100C90008F4F9F4F16C0882311F096E911C077231C
:100CA00021F09EE8872F762F05C0662371F096E825
:100CB000862F70E060E02AF09A95660F771F881FF4
:100CC000DAF7880F9695879597F90895990F000898
:100CD000550FAA0BE0E8FEEF16161706E807F9070E
:100CE000C0F012161306E407F50798F0621B730BA9
:100CF000840B950B39F40A2661F0232B242B252B2A
:100D000021F408950A2609F4A140A6958FEF811DCC
:100D1000811D089597F99F6780E870E060E008956D
:100D20009FEF80EC089500240A9416161706180603
:100D30000906089500240A941216130614060506DF
:100D40000895092E0394000C11F4882352F0BB0F70
:100D500040F4BF2B11F460FF04C06F5F7F4F8F4FD3
:100D60009F4F089557FD9058440F551F59F05F3F0E
:100D700071F04795880F97FB991F61F09F3F79F0BD
:100D800087950895121613061406551FF2CF46953F
:100D9000F1DF08C0161617061806991FF1CF8695C1
:100DA0007105610508940895E894BB2766277727A5
:100DB000CB0197F908950E94660608F48FEF089515
:100DC0000E94F3060C94A1060E94930638F00E943C
:100DD0009A0620F0952311F00C948A060C94900644
:100DE00011240C94D5060E94B20670F3959FC1F3AE
:100DF000950F50E0551F629FF001729FBB27F00DC9
:100E0000B11D639FAA27F00DB11DAA1F649F66271D
:100E1000B00DA11D661F829F2227B00DA11D621F6C
:100E2000739FB00DA11D621F839FA00D611D221F26
:100E3000749F3327A00D611D231F849F600D211D0A
:100E4000822F762F6A2F11249F5750409AF0F1F08D
:100E500088234AF0EE0FFF1FBB1F661F771F881FF6
:100E600091505040A9F79E3F510580F00C948A069E
:100E70000C94D5065F3FE4F3983ED4F386957795BE
:100E80006795B795F795E7959F5FC1F7FE2B880F9C
:100E9000911D9695879597F90895991B79E004C05F
:100EA000991F961708F0961B881F7A95C9F78095A9
:100EB000089597FB072E16F4009407D077FD09D00C
:100EC0000E946D0707FC05D03EF4909581959F4FD9
:100ED0000895709561957F4F0895AA1BBB1B51E142
:100EE00007C0AA1FBB1FA617B70710F0A61BB70B9A
:100EF000881F991F5A95A9F780959095BC01CD013F
:100F00000895EE0FFF1F0590F491E02D0994F894D9
:020F1000FFCF11
:0A0F1200010201030405081020008D
:00000001FF
